:0200000480007A
:10000000B72F0000938F0F8073900F3015A8130047
:100010000000130000001300000013000000130094
:100020000000130000001300000013000000130084
:100030000000130000001300000013000000010086
:10004000970200009382020C73905230814001416C
:100050008141014281420143814301448144014580
:100060008145014681460147814701488148014950
:100070008149014A814A014B814B014C814C014D20
:10008000814D014E814E014F814F971102009381A6
:1000900021C8170502001305E54A979503009385CB
:1000A000257201461122170502001305E53C97054C
:1000B00002009385A5450146C52817A50300130531
:1000C000657097B503009385A56F37B6ABAB130684
:1000D000B6BAD92817B103001301C16EEF60E0234F
:1000E000860293D21200F512638802008242110147
:1000F0006F00001073002030824211017300203025
:10010000711116C0F3222034E3CC02FC82421101AB
:10011000130141F806C20AC40EC612C816CA1ACC88
:100120001ECE22D026D22AD42ED632D836DA3ADCC7
:100130003EDEC2C0C6C2CAC4CEC6D2C8D6CADACC97
:10014000DECEE2D0E6D2EAD4EED6F2D8F6DAFADCA7
:10015000FEDE73252034F32510340A8601A07310C7
:10016000153492402241B2414242D2426243F243AC
:10017000025492542255B2554256D2566257F25703
:10018000064896482649B649464AD64A664BF64B33
:10019000065C965C265DB65D465ED65E665FF65F83
:1001A0001301C1077300203010C16374B50011053D
:1001B000E5BF828000000000000000000000000099
:1001C000000000000000000000000000000000002F
:1001D000000000000000000000000000000000001F
:1001E000000000000000000000000000000000000F
:1001F000197106C00AC20EC412C616C81ACA1ECC8D
:1002000022CE26D02AD22ED432D636D83ADA3EDCC6
:1002100042DEC6C0CAC2CEC4D2C6D6C8DACADECC96
:10022000E2CEE6D0EAD2EED4F2D6F6D8FADAFEDCA6
:100230009702020083A2822723A02200F322103417
:1002400096DEEF00002B1701020003212126024158
:10025000F65273901234B72200009382028873A082
:10026000023082403242C2425243E24372448254DC
:100270001255A2553256C2565257E2577258864806
:100280001649A649364AC64A564BE64B764C865C1A
:10029000165DA65D365EC65E565FE65F0961730059
:1002A0002030970202009382E22923A0120023A2A9
:1002B000220023A4320023A6420023A8520023AA2E
:1002C000620023AC720023AE820023A0920223A21C
:1002D000A20223A4B20223A6C20223A8D20223AA06
:1002E000E20223ACF20223AE020323A0120523A2F2
:1002F000220523A4320523A6420523A8520523AADA
:10030000620523AC720523AE820523A0920723A2C7
:10031000A20723A4B20723A6C20723A8D20723AAB1
:10032000E20723ACF207EF40D02E170102000321B1
:10033000E1170241F65273901234B7220000938203
:10034000028873A0023082403242C2425243E243EA
:10035000724482541255A2553256C2565257E25731
:10036000725886481649A649364AC64A564BE64B45
:10037000764C865C165DA65D365EC65E565FE65FB1
:10038000096173002030970202009382A21B83A0B0
:10039000020003A1420083A1820003A2C20083A243
:1003A000020103A3420183A3820103A4C20183A427
:1003B000020203A5420283A5820203A6C20283A60B
:1003C000020303A7420383A7820303A8C20383A8EF
:1003D000020403A9420483A9820403AAC20483AAD3
:1003E000020503AB420583AB820503ACC20583ACB7
:1003F000020603AD420683AD820603AEC20683AE9B
:10040000020703AFC20983AF820782807370043092
:10041000197106C00AC20EC412C616C81ACA1ECC6A
:1004200022CE26D02AD22ED432D636D83ADA3EDCA4
:1004300042DEC6C0CAC2CEC4D2C6D6C8DACADECC74
:10044000E2CEE6D0EAD2EED4F2D6F6D8FADAFEDC84
:100450009702020083A2820523A0220086DEEF20FD
:10046000402D17010200032161040241F6527390EE
:100470001234B72200009382028873A002308240B7
:100480003242C2425243E243724482541255A25550
:100490003256C2565257E257725886481649A649F4
:1004A000364AC64A564BE64B764C865C165DA65DD0
:1004B000365EC65E565FE65F09617300203073707A
:1004C000043001A07310453082807325403073F0F2
:1004D00043308280970700009387A7FE232EB5FE46
:1004E0002322C5FA232635F82320F5F8130505F84D
:1004F0008280411106C6EF40F00EEF10700901E551
:10050000B24041018280B24041016F2080229307B6
:1005100085007D575CC118C55CC51CC9232005003A
:1005200082802328050082805C41DCC1984798C501
:1005300098474CC38CC788C91C4185071CC1828061
:100540009041FD57130785006314F60039A83E87D4
:100550005C439443E37DD6FEDCC18CC798C54CC395
:1005600088C91C4185071CC1828018495C43EDB7CE
:10057000584114451C4914C71845544154C3D84325
:100580006314A7001845D8C32328050088437D15A8
:1005900088C382803041AE8701CE4C455841B29528
:1005A0004CC563E4E5000C414CC53E856F30102816
:1005B0008280411122C406C62A8426C2EF209010F0
:1005C0003C44635BF0025C5085CB9304440209A871
:1005D0003C44FD173CC43C446350F0025C5089CF5E
:1005E0002685EF20A0566DD5EF2080763C44FD1780
:1005F0003CC43C44E344F0FEFD573CC4EF20D00E25
:10060000EF20500C7C40635BF0021C4885CB9304C8
:10061000040109A87C40FD177CC07C406350F002B7
:100620001C4889CF2685EF2060526DD5EF2040729F
:100630007C40FD177CC07C40E344F0FEFD577CC04D
:100640002244B240924441016F20100A29C5411151
:1006500022C426C22A8406C6AE84EF20B0063440E7
:100660005C5C1840232C0402B387F6027D5670C0F0
:1006700018C430C4B386D740BA9736975CC058C404
:1006800091EC1C489DE3EF203006B2402244924496
:100690000545410182807370043001A013050401F7
:1006A000BD3513054402A535F9BF13050401EF203C
:1006B000E0498547E319F5FC913BF1B701E573701B
:1006C000043001A0011126CA4AC84EC606CE22CC6B
:1006D000B2892E89AA84A5C53305B502130555052F
:1006E000EF30807C2A8435C1930745051CC144DC6A
:1006F00023202405EF20007D34405C5C18407D56AB
:10070000B387F602232C040270C018C430C413054A
:100710000401B386D740BA9736975CC058C4C53B2E
:1007200013054402ED33EF20207C23083405228595
:10073000F2406244D2444249B249056182801305C5
:100740004005EF3060762A8401E57370043001A023
:1007500000C071BF01E57370043001A06375B5007E
:100760007370043001A0411122C409462E848145D2
:1007700006C6A93711C500DDB2402244410182807E
:100780007370043001A05D7186C6A2C4A6C2CAC03F
:100790004EDE52DC56DA5AD85ED632C6630A051CE3
:1007A0006382051C89476399F600585D8547630598
:1007B000F7007370043001A03689AE842A84EF20DC
:1007C000A05B11E5B24781C77370043001A0EF2030
:1007D000606F185C5C5C014B894BFD59130A040186
:1007E000930A44026365F70C63077919B247638182
:1007F000072463150B002808EF206048EF20C06E27
:10080000EF10C04FEF20006C7C406394370123222F
:1008100004043C446394370123240404EF20C06C97
:100820006C002808EF20C047631E051EEF2080697A
:10083000185C5C5C630CF70AEF20006BEF208068AB
:100840003C44634FF00039A85685EF20203019C191
:10085000EF2000503C44FD173CC43C446354F0007E
:100860005C50FDF323243405EF200068EF20806501
:100870007C40634FF00039A85285EF20202D19C12C
:10088000EF20004D7C40FD177CC07C406354F0009D
:100890001C48FDF323223405EF200065EF10006BA8
:1008A000054BEF202062185C5C5CE37FF7F2304080
:1008B0006305060C631F09120844A685EF30007714
:1008C0001C4434405840B6971CC463EAE70A1C5CD9
:1008D00014405850850714C41CDC5DC7130544023E
:1008E000EF20C02685476311F50AC9A8EF20C05F35
:1008F000B2455285EF204007EF20C05C3C44634F77
:10090000F00039A85685EF20602419C1EF2040443B
:100910003C44FD173CC43C446354F0005C50FDF380
:1009200023243405EF20405CEF20C0597C40634F06
:10093000F00039A85285EF20602119C1EF20404115
:100940007C40FD177CC07C406354F0001C48FDF3E4
:1009500023223405EF204059EF10405F31F17D3400
:10096000054B81B73C41E38F07E27370043001A06F
:100970007370043001A0304021E61C4085C71C5C28
:10098000585085071CDC39FBEF2000560545B64062
:10099000264496440649F259625AD25A425BB25BE7
:1009A000616182804840EF2040491C5C58502322FE
:1009B000040085071CDCE31307F279D5813CE9B715
:1009C0004844A685EF3080663C4058441440B30745
:1009D000F0403E9758C4637CD7025840BA975CC435
:1009E00009475C506306E902185C050718DCC9DF9B
:1009F000F5B54844A685EF3060633C405844144048
:100A0000B307F0403E9758C4E37CD7FCF9B75C507D
:100A1000185C79DB185C7D1718DC185C050718DC9E
:100A2000A5D76DBD22857136EF104052014585B7BF
:100A3000EF20804B0145A1BF411126C2AA841305B6
:100A4000400522C406C6EF3020462A8415CD232C4B
:100A50000502FD577CC10547410558DC3CC42322F3
:100A60000400232004002324040023260400232060
:100A7000040423089404613C13054402493C814664
:100A800001468145228501332285B24022449244A9
:100A9000410182800DC5411122C426C206C64AC04A
:100AA000032945002A84EF20602C8144630CA900AF
:100AB000B2402244268502499244410182807370EB
:100AC000043001A05C448544FD175CC4F5F3814605
:100AD0000146814522854539E1BF31CDA1C90111CA
:100AE00022CC26CA4AC852C406CE4EC68947B6840E
:100AF00032892E8A2A846399F600585D8547630FF0
:100B0000F7047370043001A0C932185C5C5CAA89D8
:100B10006366F70281444E857532F2406244268551
:100B20004249D244B249224A056182803C41C5DB38
:100B30007370043001A07370043001A0304041E2B2
:100B40001C40D5CB1C5C7D5785071CDC3C4463876F
:100B5000E7083C44854485073CC475BFBD32185C3A
:100B60005C5CAA89636DF702304079DA4844D2852B
:100B7000EF30C04B3C4058441440B307F0403E9720
:100B800058C46375D7005840BA975CC48947E39B43
:100B9000F4FA1C5CC5DB1C5CFD171CDC65B730403F
:100BA00045D24844D285EF3060483C405844144018
:100BB000B307F0403E9758C4E367D7FCD9BFDDF4D4
:100BC0000844D285EF3080461C4434405840B697E4
:100BD0001CC4E3E9E7F61C401CC4ADB75C50854477
:100BE0009DDB13054402EF10707615D5E30509F27D
:100BF000232099000DB74840EF2020242322040031
:100C000091B721CD3C4181C77370043001A01C41D4
:100C1000A1CB011122CC26CA2A844AC84EC606CED0
:100C20002E896530185C5C5CAA898144637DF7007D
:100C30001C5C7D5785071CDC3C446388E7023C4410
:100C4000854485073CC44E85B538F240624426850C
:100C50004249D244B249056182807370043001A0D8
:100C60005C41C5DB7370043001A05C5099E385449E
:100C7000D9BF13054402EF10706D75D9E30909FE61
:100C800085472320F900E5B7397106DE22DC26DA34
:100C90004AD84ED652D456D232C66302051C638A55
:100CA000051AB68AAE892A84EF20000D11E5B247F5
:100CB00081C77370043001A0EF20C0201C5C6392D8
:100CC0000714B247638E070A2808EF10507BFD54C3
:100CD00013094402130A0401EF200021EF1000025F
:100CE000EF20401E7C4063949700232204043C4480
:100CF0006394970023240404EF20001F6C0028084D
:100D0000EF10107A63130518EF20C01B1C5CADCFE9
:100D1000EF20801DEF20001B3C44634FF00039A8FA
:100D20004A85EF10B06219C1EF2080023C44FD17E4
:100D30003CC43C446354F0005C50FDF324C4EF20F9
:100D4000A01AEF2020187C40634FF00039A852858C
:100D5000EF10D05F19C1EF10B07F7C40FD177CC051
:100D60007C406354F0001C48FDF364C0EF20C017C2
:100D7000EF10C01DEF2000151C5CC1E7B247A9FFB2
:100D8000EF208016014555A0EF2000161C40DDC75E
:100D9000B2454A85EF10503DEF20C0123C44634FEE
:100DA000F00039A84A85EF10705A19C1EF10507A37
:100DB0003C44FD173CC43C446354F0005C50FDF3DC
:100DC00024C4EF206012EF20E00F7C40634FF0005E
:100DD00039A85285EF10905719C1EF1070777C40F9
:100DE000FD177CC07C406354F0001C48FDF364C0D8
:100DF000EF20800FEF10801531C9EF20A00C1C5C94
:100E0000B5DFCE8522854444EFF0CFF8639C0A0419
:100E10001C5C1840FD171CDC01E7EF20601148C086
:100E20001C48A1EFEF20400C0545F2506254D2540B
:100E30004259B259225A925A21618280EF20800889
:100E40004840EF107075EF20200A99B7EFF00FDCE3
:100E50006DB73C41E38707E47370043001A0737001
:100E6000043001A05C5044C4D5DF13054402EF10E8
:100E7000F04D4DD9EFF08FD975B713050401EF1080
:100E8000F04C8547E310F5FAF5B72285EFF06FF2E5
:100E9000EF10C00B014551BF1DC9411122C44AC00A
:100EA00006C626C244412E892A84EF10306C638323
:100EB000A40281464A8681452285F933854763002D
:100EC000F502B2402244924402494101828073708B
:100ED000043001A05C44054585075CC4DDB75C4473
:100EE00085075CC4F9BF15CDADC9011122CC26CA56
:100EF0004AC84EC652C42A8406CE3289AE89EFF063
:100F0000CFDC1C5C2A8A814485E35285EFF08FDBBD
:100F1000F240624426854249D244B249224A0561E0
:100F200082807370043001A0304001CE4C445C409C
:100F3000B2954CC463E4F5000C404CC44E85EF30D0
:100F4000E00E1C5C7D57FD171CDC7C40638CE700C9
:100F50007C40854485077CC04DBF3C41D9D7737028
:100F6000043001A01C4899E3854445B713050401EA
:100F7000EF10D03D75D9E30909FE85472320F9001C
:100F8000E5B721C93C41A1CDA1CB011122CC26CA94
:100F90004AC852C42A8406CE4EC62E8AEFF0EFD23B
:100FA0001C5C2A89814491CB8329C400D285228587
:100FB000EFF04FDE8544232634014A85EFF08FD0D1
:100FC000F240624426854249D244B249224A056130
:100FD00082807370043001A07370043001A0EDDFD3
:100FE0007370043001A001E57370043001A0411159
:100FF00022C42A8406C6EF10F06C005CEF10D06E9D
:10100000B240228522444101828001E573700430A0
:1010100001A0411106C622C42A84EF10B06A1C5CEC
:10102000405C1D8CEF10506C2285B240224441017F
:10103000828019C1085D82807370043001A01DCDCB
:101040009787030093870774D843630CE502D8475A
:10105000630CE504D84B6307E504D84F6302E5044D
:10106000D853630DE502D8576308E502D85B6303E4
:10107000E502D85F630EE5006F20307573700430B1
:1010800001A001470E07BA9723A007006F20F07355
:101090001D47CDBF1947FDB71547EDB71147DDB760
:1010A0000D47CDB70947F9BF0547E9BF68458280BD
:1010B0006CC5828003450505828009C5085D13352E
:1010C000150082807370043001A019C51C5D485D55
:1010D0001D8D1335150082807370043001A0978731
:1010E00003009387276A984305C3984705C7984B21
:1010F00005C7984F05C7985305C7985705C7985B0C
:1011000015C7985F15C3828001470E07BA978CC335
:10111000C8C382800547D5BF0947C5BF0D47F5B78E
:101120001147E5B71547D5B71D47C5B71947F1BFF3
:101130009787030093870765D8436308E502D8477C
:10114000630BE502D84B630AE502D84F6309E50259
:10115000D8536308E502D8576307E502D85B6308F4
:10116000E502D85F6303A702828001470E07BA97A2
:1011700023A0070082800547D5BF0947C5BF0D479B
:10118000F5B71147E5B71547D5B71D47C5B7194797
:10119000F1BF411122C426C24AC02A8406C6AE84C9
:1011A0003289EF1030527840FD576314F700232244
:1011B00004043844FD576314F70023240404EF109B
:1011C000B0521C5C99E74A86A68513054402EF10CD
:1011D000B00CEF10304F3C44635BF0025C5085CBA9
:1011E0009304440209A83C44FD173CC43C446350AA
:1011F000F0025C5089CF2685EF1050156DD5EF10A9
:1012000030353C44FD173CC43C44E344F0FEFD57FC
:101210003CC4EF10704DEF10F04A7C40635BF0026D
:101220001C4885CB9304040109A87C40FD177CC0B1
:101230007C406350F0021C4889CF2685EF101011C6
:101240006DD5EF10F0307C40FD177CC07C40E3444E
:10125000F0FEFD577CC02244B24092440249410155
:101260006F10904805C579714ECE52CC06D63E8A95
:1012700022D426D24AD056CA5AC85EC662C4A547EE
:10128000BA8963F8E7007370043001A0737004300A
:1012900001A0AA8AAE843289B68B428B63090822E8
:1012A00013050006EF2050402A84630D05200A092B
:1012B000232865034A869305500A5A85EF20106556
:1012C00003C704001C587119230AE40203C7040071
:1012D0003E991379C9FF79C783C71400A30AF402A2
:1012E00083C71400E1C383C72400230BF40283C720
:1012F0002400CDCB83C73400A30BF40283C7340092
:10130000D5C383C74400230CF40283C74400D9CB60
:1013100083C75400A30CF40283C75400C1C783C71A
:101320006400230DF40283C76400ADCF83C774004B
:10133000A30DF40283C77400B5C783C78400230ECE
:10134000F40283C78400B9CF83C79400A30EF402CC
:1013500083C79400A1CB83C7A400230FF40283C7E3
:10136000A400A9C383C7B400A30FF40283C7B400C9
:1013700095CB83C7C4002300F40483C7C4009DC376
:1013800083C7D400A300F40483C7D40081CF83C7EC
:10139000E4002301F40483C7E40089C783C7F40091
:1013A000A301F404130B44005A85A301040423266B
:1013B000340323283405232A0404EFF08F96130501
:1013C0008401EFF00F96A947B3873741232C04041B
:1013D00000C81CCC40D023220404232E04045E86C3
:1013E000D6854A85EFF00F8F08C063040A002320DA
:1013F0008A007370043017F9010013096909832703
:10140000090097F401009384640A91C798409C40B6
:101410007C4385077CC317F70100130727081C438B
:10142000850797F6010023ABF6069C40D5CB8327B2
:10143000090017FA0100130AAA1889EB9C40DC572F
:1014400063E6F90097F7010023A2870697F70100EA
:1014500093870703984397F601009386A6035C548D
:101460009442050717F60100232CE60038C463F602
:10147000F60017F70100232FF7005147B387E70263
:10148000DA853305FA00EFF02F8A8327090081C738
:101490009C40FC43BDE383270900054499C79C4059
:1014A000DC5763F43701EFE07FF62285B250225417
:1014B00092540259F249624AD24A424BB24B224CF0
:1014C000456182805A85EF2050307D54F9BF131555
:1014D0002600EF20701D2A8BE31405DC7D54F1B744
:1014E00097F7010023A487FC184385476301F7029F
:1014F00017FA0100130ACA0C91BF984094407C432C
:10150000FD177CC3FC42C1FB7360043069B7814A9C
:1015100017FA0100130ACA0A514CA94B33858A03F2
:10152000850A5295EFE0BFFEE39A7AFF97FB010030
:10153000938B8B155E85EFE09FFD97FA0100938AF0
:10154000EA155685EFE0BFFC17F5010013054516B7
:10155000EFE0FFFB17F501001305C516EFE03FFBB9
:1015600017F5010013054517EFE07FFA97F7010023
:1015700023AC77F397F7010023A657F3C1BD4111C0
:1015800022C406C626C24AC02A847370043097F467
:1015900001009384E4EF9C40F9E311E497F7010024
:1015A0009387C7F08043130944004A85EFE05FFC4E
:1015B0001C5489C713058401EFE09FFBCA8517F50A
:1015C000010013052510EFE03FF697F70100938720
:1015D00027ED984397F70100938787EA9C43050717
:1015E00097F6010023AEE6EA9840850797F60100DA
:1015F00023A8F6E801CB97F70100938727EB9843E0
:10160000784349EF9C40B1C797F70100938707EAF9
:101610009843630F870873700430984039EB17F7CD
:101620000100130767E814439442A5E27D5797F63B
:10163000010023A5E6E4984009CF9843784311CBF5
:10164000984394437C43FD177CC3FC4299E3736049
:101650000430B2402244924402494101828097F70B
:1016600001009387A7E498439C437C4385077CC390
:101670002DB794439843F8420507F8C217F70100C5
:10168000130787E214439442D5D21843584758476A
:10169000584397F6010023A3E6DE71BF98439443B5
:1016A0007C43FD177CC3FC42B1FF7360043099BFDB
:1016B00097F70100938747DC9C4381C77370043020
:1016C00001A02244B2409244024941016FE01FD47C
:1016D00041C517F70100130767DD14438147638B8A
:1016E000A606411106C622C426C27370043097F6BE
:1016F00001009386E6D99C4291C710431C437C426B
:1017000085077CC29C42AA84404981C71C43FC4394
:10171000B9E797F70100938727D99C43638B870428
:1017200097F70100938707D89C436384870497F752
:101730000100938767FA6309F40297F70100938722
:1017400067F86301F4028547B240224492443E8523
:10175000410182803E8582807370043001A0EF4099
:10176000303145BF9147CDB79C5493B717008907D7
:10177000E1BF8947D1BF7370043097F701009387A9
:1017800027D1984309EF15C59C43485581CB97F75E
:1017900001009387A7D19843784315E3828017F718
:1017A00001001307A7D014431843F8420507F8C2F5
:1017B00061FD17F70100130767CF0843F1B798439E
:1017C00094437C43FD177CC3FC42E9FB7360043007
:1017D0008280411122C42A8406C6EFE01FCF11E4A3
:1017E00097F70100938787CC80434054EFE09FCD6B
:1017F000B2402285224441018280A54763F5B700AB
:101800007370043001A0011122CC06CE26CA4AC84A
:101810004EC652C42A847370043017F901001309AC
:1018200029C783270900D5EF79C43C486389F508A7
:1018300017F70100130787C763FCB7001443638DD4
:10184000860C18434457B3B4950093C4140029A0E0
:101850000443818C93B4140058546384E70A1C4CED
:101860002CC863C60700A947B385B7400CCC9317B3
:101870002700BA97584897F90100938969D48A07D5
:10188000CE97631BF702130A44005285EFE05FCE48
:1018900017F70100130707C05C5418436376F7007D
:1018A00017F701002328F7BE5147B387E702D28517
:1018B0003385F900EFE05FC799C0EFE03FB58327BC
:1018C000090081CB97F70100938747BE9C43FC43F7
:1018D0009DEBF2406244D2444249B249224A05613A
:1018E000828097F70100938767BC98439C437C43B1
:1018F00085077CC31DF897F70100938727BB8043BA
:101900002DB74CD4A9BF6244F240D2444249B249F7
:10191000224A05616F40D01581443DBF25C10111A8
:1019200026CA97F40100938464B89C4006CE22CC6A
:101930004AC84EC6638DA7027370043017F90100C0
:10194000130909B58327090091C798409C407C433F
:1019500085077CC3584997F701009387E7D763024F
:10196000F7028327090081C79C40FC43A5EBF240A6
:101970006244D2444249B2490561828073700430A6
:1019800001A01C5517F70100130787D2E38BE7FC72
:10199000E9FB930945002A844E85EFE07FBD17F7E8
:1019A0000100130727AF5C5418436376F70017F75D
:1019B00001002321F7AE5147B387E70217F5010075
:1019C000130505C0CE853E95EFE01FB69C405854E8
:1019D000DC57E368F7F8EFE07FA361B76244F240B9
:1019E000D2444249B24905616F40900815CD0111BA
:1019F00022CC26CA4AC82A8406CE4EC6EFE0FFACE7
:101A0000584897F70100938727CD2A8981446300BE
:101A1000F7024A85EFE01FABF24062442685424957
:101A2000D244B249056182807370043001A01C5415
:101A300017F501001305C5C7E38DA7FCF9FB97F760
:101A40000100938767A39C43A9EB97F70100938755
:101A5000E7A59C43445493094400DC574E85B3B436
:101A6000F400EFE0FFB017F701001307A7A25C54E2
:101A7000184393C414006376F70017F70100232B73
:101A8000F7A05147B387E70217F50100130545B3E7
:101A9000CE853E95EFE05FA9ADBF93058401EFE0F1
:101AA000BFA885BF0111056506CE22CC26CA4AC84B
:101AB0004EC652C456C25AC0EF20003F630E051AEC
:101AC000AA8413050006EF20203E2A84630A051C21
:101AD00005669305500A04D92685EF202063045833
:101AE0008567F117BE94B7474C4593879744130A0F
:101AF00044005CD85285230C0402A301040423266D
:101B0000040223280404232A0404EFE09FA1130500
:101B10008401EFE01FA1A947232C0404F19800C819
:101B20001CCC40D023220404232E04040146971524
:101B300000009385E5B12685EFE0DF9908C073705A
:101B4000043017F901001309A9948327090097F4B9
:101B500001009384A49591C798409C407C438507DD
:101B60007CC317F70100130767931C43850797F69B
:101B7000010023A5F6929C40C9C38327090097F969
:101B800001009389E9A381EB9C40DC5789E797F733
:101B9000010023AD879097F701009387678E9843E4
:101BA00097F601009386068F5C549442050717F65A
:101BB00001002327E68C38C463F6F60017F701000E
:101BC000232AF78C139527003E950A05D2854E955A
:101BD000EFE09F958327090081C79C40FC43DDE728
:101BE0008327090091C39C40EF10F04985476305A6
:101BF000F50C59E17370043001A097F7010023A799
:101C0000878A1843854797F901009389699BE314F4
:101C1000F7F8CE8A17FB0100130B0BA75685D10AE4
:101C2000EFE0FF8EE31C5BFF17F501001305C5A570
:101C3000EFE0FF8D97FA0100938A4AA65685EFE000
:101C40001F8D17F501001305A5A6EFE05F8C17F5B2
:101C50000100130525A7EFE09F8B17F50100130581
:101C6000A5A7EFE0DF8A97F7010023AF678397F717
:101C7000010023A9578305B7F2406244D244424988
:101C8000B249224A924A024B0561828098409440B0
:101C90007C43FD177CC3FC42A1F77360043089B715
:101CA0006244F2404249B249224A924A024B268596
:101CB000D24405616F20603173700430FD5717E71F
:101CC0000100232DF77A624497E7010023A2A77C45
:101CD000F240D2444249B249224A924A024B97E723
:101CE000010023AB077A05616FE0AFDB737004304E
:101CF00097E7010023AE07786FE0EFE817E70100F0
:101D0000130787771C4385071CC3828073700430D8
:101D100097E701009387C777984305E317E701002A
:101D20001307877708439C4381CB97E7010093878C
:101D3000E7779843784301EF828017E701001307A4
:101D4000E77614431843F8420507F8C2C1BF984329
:101D500094437C43FD177CC3FC42F9FF736004305D
:101D60008280411106C622C4EFE02FF697E70100FA
:101D7000938787728043EFE0EFF4B24022852244DC
:101D80004101828097E701009387477188438280F1
:101D9000797106D622D426D24AD04ECE52CC56CA1B
:101DA0005AC85EC697E701009387076D9C43B1EF61
:101DB00017E701001307476E1C43850797E60100EC
:101DC00023ACF66C832A0700638F0A0697E70100AD
:101DD0009387C76A9C43814463F1FA0897E901003D
:101DE0009389097E17EA0100130A4A6C83270A00C7
:101DF0008546D85793172700BA978A07BE9983A7B5
:101E0000090063FFF600854421A897E70100938746
:101E1000E7679C438144850717E701002328F7669D
:101E200097E70100938747669C4391C38544B2506E
:101E30002254268502599254F249624AD24A424BB0
:101E4000B24B4561828017E401001304E4651C4035
:101E50009C43DDC37370043001A017E40100130438
:101E6000A46497E901009389A97517EA0100130A90
:101E7000EA6317EB0100130BEB611C409C43B5C3F5
:101E80001C40DC4703A9C70083274900930B490086
:101E90005E8563EEFA04EFE0AFED83278902130558
:101EA000890199C3EFE0CFEC8327C90203270B0018
:101EB000DE85139527003E950A054E956376F7005B
:101EC00017E701002328F75CEFE00FE683270A00FD
:101ED0000327C902DC57E362F7FA1C4085449C43A0
:101EE000C5F3FD5717E70100232AF75801B717E795
:101EF00001002325F758DDBD17E701001307875AB6
:101F00001C40184397E6010023A0E65A17E701009A
:101F1000232AF75897E701009387C7569C43850704
:101F200017E701002320F7561C409C4399E7FD5713
:101F300017E701002324F75451BD1C40DC47DC4760
:101F4000DC4317E70100232BF75249B597E701005F
:101F500093878752984301E77370043001A0011101
:101F600006CE22CC26CA4AC84EC652C456C25AC051
:101F70007370043097E4010093848451984061EBBE
:101F800098437D1797E6010023A8E64E9C43D9EBC2
:101F900097E70100938787509C43C9C797EA0100E0
:101FA000938A0A6217EA0100130ACA4E17E9010070
:101FB0001309C94F854919A83385EA00EFE0CFD648
:101FC000832709005854DC576379F70483A70A0F65
:101FD000C1CF83A7CA0FC04713058401EFE04FD9D3
:101FE000130B44005A85EFE0AFD85C5483260A00F7
:101FF000DA85139527003E950A052A875695E3FD55
:10200000F6FA17E701002327F748EFE0EFD183271F
:1020100009005854DC57E36BF7FA97E7010023A552
:1020200037476DB701449C4081CB97E70100938708
:10203000E7479C43FC4395E72285F2406244D24443
:102040004249B249224A924A024B0561828017E70F
:1020500001001307A74514431843F8420507F8C2C7
:1020600005B7EF40E020C9BF17E4010013040442A4
:102070001C4095C31C40054999CF193B09C597E7FA
:10208000010023A327411C40FD1717E70100232F60
:10209000F73E1C40FDF397E701009387E73E984326
:1020A0008547E311F7F8EFE06FB60544ADBF11CDFA
:1020B00081E57370043001A017E701001307C73BE7
:1020C0001C4399C77370043001A07370043001A0E1
:1020D000411122C406C614431841850617E60100C3
:1020E000232CD63897E601009386063B94423304AE
:1020F000B70000C163F7E602637FE40063FD86007A
:1021000097E701009387873A88431105EFE04FC6B0
:102110002285EF40A00F1D3D01C9B240224441017C
:102120008280E36FE4FCD9BF2244B24041016FE0FA
:10213000EFAD11C917E70100130707341C4391C71E
:102140007370043001A06FE06FAC411106C622C469
:102150001843AA87050797E6010023AFE63097E604
:1021600001009386A63417E701001307E7321843EE
:1021700088423304F7001105EFE08FBF2285EF405E
:10218000E008E93311E52244B24041016FE00FA8B5
:10219000B240224441018280411122C406C697E721
:1021A00001009387672D9C430144850717E70100D1
:1021B0002324F72C97E701009387472E9C4363E085
:1021C000F51217EE0100130E6E4B97E20100938299
:1021D000623E01440147854F1303500A21A0311E7E
:1021E000638DC20B83278EFFBA86F5DB8327CEFF74
:1021F000DC43232EFEFE638AC70F03AFC700DC4318
:102200002A97814E232EFEFE6385C70783A8C70049
:1022100093874803232017015CC383A788042326E0
:10222000F7011CC783A7C8021CCB83A70805232C72
:1022300007005CCB03A8080383470800639067048A
:10224000C287850783C60700B3850741E38B66FE17
:102250008981C205C181231EB700850E13070702BD
:1022600063061F038327CEFFDC43232EFEFEE39F7E
:10227000C7F983274E00232EFEFE49BF8145231E4A
:10228000B700850E13070702E31E1FFD7694131790
:102290005400311EBA86E397C2F597E70100938791
:1022A000A72003AE070083270E00639D070E97E764
:1022B00001009387271F03AE070083270E00639258
:1022C000071817EE0100130EAE2F83274E109DE363
:1022D00083278E116395072019C223200600BD3184
:1022E0002285B24022444101828083274E00232E62
:1022F000FEFE21B783278E1017EF0100130F0F3D4D
:10230000DC4317E701002321F73C6380E73383A216
:10231000C700DC43AA96814E17E701002326F73A4F
:10232000914F1303500A6388E70783A8C700938778
:10233000480323A01601DCC283A7880423A6F60164
:102340009CC683A7C8029CCA83A7080523AC0600C5
:10235000DCCA03A80803834708006391672AC28781
:10236000850703C70700B3850741E30B67FE93D7D3
:102370002500C207C183239EF600850E93860602C0
:102380006386122983278E10DC4317E70100232D73
:10239000F732E39CE7F983270E1117E701002325A5
:1023A000F73261B783274E00130F8E00D4432322E8
:1023B000DE006388E629B307E500D84283A2C600A1
:1023C000814E2322EE00894F1303500A6306EF0665
:1023D0008328C7001387480323A01701D8C303A786
:1023E000880423A6F70198C703A7C80298CB03A7C0
:1023F000080523AC0700D8CB03A80803034708004F
:102400006318671C4287050783460700B305074129
:10241000E38B66FE13D7250042074183239EE70026
:10242000850E93870702638D121B83264E00D842C8
:102430002322EE00E31EEFF80327CE002322EE0056
:1024400041BF83274E00130F8E00DC432322FE0082
:102450006384E71F83A2C700DC43AA96814E232230
:10246000FE00894F1303500A6306FF0683A8C700C6
:102470009387480323A01601DCC283A7880423A600
:10248000F6019CC683A7C8029CCA83A7080523AC93
:102490000600DCCA03A80803834708006396671098
:1024A000C287850703C70700B3850741E30B67FEB3
:1024B00093D72500C207C183239EF600850E93861D
:1024C0000602638B120F83274E00DC432322FE009B
:1024D000E31EFFF88327CE002322FE0041BF83279F
:1024E000CE1197EE0100938EAE1FDC4317E701007B
:1024F0002326F71E6384D71383AFC700DC4333075B
:10250000D500014397E6010023AAF61C0D4F89422E
:102510009308500A6387D707C8479307450308C342
:102520005CC33C452326E7011CC75C551CCB1C55EE
:1025300099C3232657003C49232C07005CCB032872
:1025400005038347080063951705C287850783C67F
:102550000700B3850741E38B16FF93D72500C20719
:10256000C183231EF700050313070702638AAF0226
:102570008327CE11DC4397E6010023A1F616E39DE5
:10258000D7F983274E1297E6010023A9F61469B7FD
:102590008147231EF700050313070702E39AAFFCE8
:1025A0001A94E31C06D225BB8147239EF600850EB4
:1025B00093860602E39912F117EE0100130E4E0006
:1025C00083274E10769493165400E38307D01DB3EF
:1025D0000147239EE700850E93870702E39712E5E4
:1025E00097E70100938707EC03AE070076949316F4
:1025F000540083270E00E38607CCA1B58147239EB4
:10260000F600850E93860602E39E12D783278E116D
:10261000769493165400E38107CCD1B583274E12EC
:1026200017E70100232CF70AC1BD83270E1117E716
:102630000100232BF708E1B98327CE002322FE00F7
:1026400011BD8326CE002322DE00B5B3797126D2D8
:102650004AD04ECE52CC56CA5AC85EC606D622D4EE
:1026600097E90100938949E117E90100130949F548
:1026700017EA0100130ACAE197EA0100938A0AE304
:1026800097EB0100938B8BE197E40100938444E185
:10269000054B21A883A7090003244910850717E7E4
:1026A0000100232BF7DC5D3011E89C40E5F7832720
:1026B0000900E37CFBFEEFD07FD5C5BF737004300B
:1026C00083270A00B9E383270911C0471305440093
:1026D000EFD01FEA83A70B00FD1717E70100232F98
:1026E000F7DA9C40FD1717E70100232BF7DA832761
:1026F0000A0089C783A70A00FC4385E30858EF1046
:10270000D00C2285EF10700C4DB703A70A0083A7E9
:102710000A007C4385077CC37DB703A70A0083A614
:102720000A007C43FD177CC3FC42E9FB7360043064
:10273000F1B797E70100938727D49C43DDE341116C
:1027400006C697E7010023A107D417E70100130786
:10275000E7D51C43B7A6A5A59386565A9C5B8C4328
:10276000639BD500D0436318B60094476395C600B9
:10277000DC476388D70008430C4393854503EF206B
:10278000D00197E601009386E6D0904217E701005A
:10279000130707E311A89C42B9CB9C42FD1717E62B
:1027A00001002329F6CE904293172600B2978A079C
:1027B000BA979C43EDD3904293172600B2978A07AD
:1027C000B305F700D441A107BA97D442D4C16383BB
:1027D000F602DC46B24017E701002329F7CC41019D
:1027E0008280854717E701002320F7CA8280737033
:1027F000043001A0D1473306F602D442329754C3C5
:10280000C9BF01114AC806CE22CC26CA4EC62A89A3
:102810007370043097E40100938484C79C4017E4EC
:1028200001001304A4C8D9E76314090003290400B4
:10283000930949004E85EFD0BFD38327890289C70A
:1028400013058901EFD0DFD2CE8517E5010013050E
:10285000A5E8EFD07FCD9C4081C71C40FC43ADE391
:102860001C40638B27079C409DCF737004309C40B5
:10287000C1EB97E70100938727C39843184325EBE3
:10288000FD5717E70100232BF7BE9C4089CF1C4062
:10289000FC4391CB184014407C43FD177CC3FC42A1
:1028A00099E373600430F2406244D2444249B24931
:1028B0000561828018401C407C4385077CC3ADB70E
:1028C000184014407C43FD177CC3FC42D1FB73606D
:1028D00004301C40E39927F99C40A1C397E701000D
:1028E000938787B99C43ADCB7370043001A09C43A0
:1028F000DC47DC47DC4317E701002321F7B871B759
:1029000018401C407C4385077CC397E701009387F0
:10291000A7B9984318432DD7D9BF97E701009387EC
:10292000E7B717E701001307A7C99C4303278711DF
:10293000631DF700F240624497E7010023A807B641
:10294000D2444249B249056182806244F240D24495
:102950004249B2490561F1BB6244F240D244424966
:10296000B24905616FD09FAA3DC9411126C297E4C3
:1029700001009384A4B34AC02E898C4006C622C4A9
:10298000E105EFD0FFBB88401105EFD07FBEFD57BA
:10299000630AF90497E70100938707B080439840E2
:1029A0009C434A9440C3636CF40497E70100938707
:1029B000A7AF88438C409105EFD09FB897E70100FF
:1029C0009387C7AB9C436376F40097E7010023A786
:1029D00087AAB24022449244024941018280737026
:1029E000043001A08C402244B2409244024917E5D1
:1029F0000100130565CE910541016FD0FFB297E745
:102A00000100938727AA884322448C40B240924415
:102A10000249910541016FD0BFB211C997E701008A
:102A2000938787A59C4399E77370043001A0737066
:102A3000043001A0411126C297E40100938404A749
:102A40009840AE878C40B7060080D58F06C622C45A
:102A50001CCFE1053284EFD03FAD88401105EFD0A7
:102A60003FB1FD57630EF40097E701009387C7A2BB
:102A70008843B24092442295224441016F3000794C
:102A80008C402244B240924417E501001305C5C4AE
:102A9000910541016FD05FA925CD411126C297E470
:102AA00001009384A4A04AC02E898C4006C622C48B
:102AB000E1053284EFD05FA788401105EFD05FAB0E
:102AC0008547630AF40497E701009387E79C8043F6
:102AD00098409C434A9440C3636CF40497E7010018
:102AE0009387879C88438C409105EFD07FA597E71B
:102AF00001009387A7989C436376F40097E7010051
:102B000023AE8796B240224492440249410182801A
:102B10007370043001A08C402244B24092440249B8
:102B200017E50100130545BB910541016FD0DF9FFB
:102B300097E7010093870797884322448C40B2406F
:102B400092440249910541016FD09F9F411106C6F1
:102B500022C426C25C45C04735CC93048401268537
:102B6000EFD01FA197E70100938707919C43B5E73A
:102B7000930444002685EFD0BF9F97E70100938719
:102B8000679158549C4363F6E70097E7010023A33D
:102B9000E79093172700BA978A0717E501001305F6
:102BA00025A2A6853E95EFD03F9897E70100938731
:102BB000E78F9C4358540145DC5763F8E70085478D
:102BC00017E701002322F78C0545B24022449244C6
:102BD000410182807370043001A0A68517E50100D1
:102BE000130505ADEFD05F94C9B797E70100938750
:102BF000A7889C4381E77370043001A0411106C689
:102C000022C426C2B70700804045CD8F1CC12DC409
:102C1000EFD01F96930444002685EFD07F9597E769
:102C200001009387278758549C4363F6E70097E792
:102C3000010023A1E78693172700BA978A0717E5B3
:102C400001001305E5973E95A685EFD0FF8D97E728
:102C500001009387A7859C4358540145DC5763F8CE
:102C6000E700854717E701002320F7820545B240BA
:102C700022449244410182807370043001A011CD3E
:102C800097E7010093870780984397E701009387B0
:102C9000A7809C4318C15CC182807370043001A07E
:102CA00055C1D1CD411106C622C42A8773700430A4
:102CB00097D801009388C87D83A7080091CB97D748
:102CC00001009387A77E94439C43FC428507FCC286
:102CD00017D301001303437C9C4103260300FD56D8
:102CE0000144638FD70217DE0100130EAE7903256E
:102CF0000E000328070054436305A80005446371D0
:102D0000D6023308D6400544637CF80003250E0044
:102D1000918F03260300B6979CC108C350C301449A
:102D200083A7080081CB97D70100938727789C431E
:102D3000FC4381EF2285B2402244410182807370BE
:102D4000043001A07370043001A0EF306052DDB791
:102D5000854717D701002329F772828019C168457A
:102D600082800145828011C16CC5828097D70100A5
:102D70009387C7738843828097D7010093874771F1
:102D80009C43054589CB97D701009387E76E88431D
:102D9000133515000605828031CD011126CA97D45E
:102DA00001009384A4709C4006CE22CC4AC84EC633
:102DB0005855DC576379F7021C4D63C707009C40E8
:102DC000D457A947958F1CCD93172700BA97584918
:102DD00017D901001309C97E8A07CA97630DF70046
:102DE0009C40DC575CD5F2406244D2444249B2492F
:102DF000056182808280930945002A844E85EFD048
:102E00002FF79C4017D701001307C7681843DC57FA
:102E10005CD46376F70017D70100232DF76613956E
:102E200027003E9562440A05F240D244CE854A9579
:102E3000B249424905616FD02FEF19CD411106C645
:102E400022C426C297D70100938747668043630751
:102E5000A4007370043001A0014582807C4881E7A2
:102E60007370043001A054543848FD177CC8638344
:102E7000E60099C70145B240224492444101828054
:102E8000930444002685EFD0AFEE3C4817D70100ED
:102E900013074760144329471D8F5CD418CC63F691
:102EA000F60017D701002327F75E5147B387E702E3
:102EB00017D501001305C570A6853E95EFD0CFE666
:102EC000054555BF7370043097D701009387475C61
:102ED0009C4391CB97D701009387475D98439C43D0
:102EE0007C4385077CC3828097D701009387475A2C
:102EF0009C438DC397D701009387475B98437843E2
:102F000011CB984394437C43FD177CC3FC4299E367
:102F100073600430828097D70100938727599043CC
:102F200094439843A947D456084E958F1CCF82806E
:102F300097D7010093878757984309C79443F84A66
:102F40000507F8CA8843828079714AD006D622D410
:102F500026D24ECE2A897370043097D40100938410
:102F600024539C4017D4010013044454BDE31C4077
:102F7000BC4F89E71C400547F8CFD1E19C4081C791
:102F80001C40FC43F1EB737004309C408DEF1C40FF
:102F9000A84F11C5630409021C4023AC07041C4060
:102FA00023AE07049C4081C71C40FC438DEBB2500C
:102FB000225492540259F2494561828018403C4F94
:102FC000FD173CCFE9BF18401C407C4385077CC3FC
:102FD0007DBF18401C407C4385077CC349BF184017
:102FE00014407C43FD177CC3FC42F1F37360043052
:102FF000B250225492540259F249456182800840ED
:103000002EC61105EFD0CFD6B245FD576380F50629
:1030100097D701009387474883A9070018409C432E
:10302000AE992322370163ECF90497D70100938707
:10303000A74788430C409105EFD08FD097D7010068
:103040009387C7439C4363F6F90097D7010023A7F2
:103050003743EFD0AFBB1DB7184014407C43FD177A
:103060007CC3FC428DF37360043031BF0C4017D534
:103070000100130565669105EFD00FCBD9BF97D737
:1030800001009387274288430C409105EFD04FCB36
:10309000C9B779714AD04ECE06D622D426D252CCA8
:1030A0002E89B2897370043097D401009384443E12
:1030B0009C4017D401001304643FF9EF184089477E
:1030C000784F630CF7001C401345F5FFB84F798D1E
:1030D000A8CF1C400547F8CFADE69C4081C71C40F7
:1030E000FC43F5E3737004309C40B1E7638609004C
:1030F0001C40BC4F23A0F900184085470145784F7C
:10310000630BF7001C401349F9FF0545B84F3379AD
:10311000E90023AC27051C4023AE07049C4081C76F
:103120001C40FC43C1E3B250225492540259F2496C
:10313000624A4561828018401C407C4385077CC3FD
:1031400075B7084036C61105EFD08FC2B246FD579D
:103150006385F60897D701009387073403AA070011
:1031600018409C43369A232247016363FA0897D795
:1031700001009387673388430C409105EFD04FBC23
:1031800097D701009387872F9C436370FA0697D7E0
:10319000010023A5472F91A818401C407C438507B8
:1031A0007CC329BF184014407C43FD177CC3FC42FC
:1031B000BDFB73600430B250225492540259F2495C
:1031C000624A45618280184014407C43FD177CC3ED
:1031D000FC4289FB7360043031B70C4017D5010005
:1031E0001305854F9105EFD02FB4EFD02FA2F5B581
:1031F00097D701009387072B88430C409105EFD0A8
:103200002FB4E5B751C1411106C622C426C24AC037
:103210007370043097D40100938484279C40B9EBE9
:1032200099C23C4D9CC2B2878946704D74CD2E87A1
:103230002A846386D70663FCF6048D456387B7004E
:1032400091456395B7006300D60C38CC8547630F72
:10325000F60405449C4081CB97D70100938707254E
:103260009C43FC43A9E32285B24022449244024994
:103270004101828097D701009387472398439C435D
:103280007C4385077CC369BF7370043001A0854609
:10329000E39ED7FA3C4D33E7B70038CD45BF3C4DF0
:1032A00085073CCD65B7EF20B07C75BF130944009E
:1032B0004A85EFD0EFAB17D701001307A71D5C5469
:1032C00018436376F70017D701002325F71C5147F1
:1032D000B387E70217D501001305852ECA853E95F1
:1032E000EFD08FA41C5481C77370043001A097D70E
:1032F00001009387A71B9C435854DC57E3FBE7F47A
:10330000EFD0CF90B9B70144B1B739CD011122CC7C
:1033100026CA4AC84EC652C456C206CEBA89368A92
:10332000B2842E892A84EFD04F9AAA8A63050A00B4
:103330003C4C2320FA00784C89477CCC6389F4020A
:1033400063F4970C8D466387D40091466396D4004E
:10335000630AF70A232C24058547631EF7061C54CD
:1033600099CB7370043001A07370043001A03C4C01
:1033700085073CCCD5B797D701009387E70F9C43CF
:10338000ADEB930444002685EFD08F9E17D7010044
:10339000130747105C5418436376F70017D70100F2
:1033A000232AF70E5147B387E70217D5010013050B
:1033B0002521A6853E95EFD02F9797D701009387BB
:1033C000E70E9C435854DC5763F7E7006385090018
:1033D000854723A0F90005445685EFD0AF8E22859E
:1033E000F2406244D2444249B249224A924A0561BB
:1033F00082809305840117D501001305652BEFD05A
:10340000AF9265BF0144C9BF8547E397F4F43C4CD4
:1034100033E92701232C240581B74DC1011122CCAA
:1034200026CA2A844AC806CE4EC6AE84EFD0EF899B
:103430008947744C7CCC3C4C05472A8985073CCC99
:103440006395E6061C5481C77370043001A097D7BA
:103450000100938767029C43ADE7930944004E85C2
:10346000EFD00F9117D701001307C7025C54184320
:103470006376F70017D70100232EF7005147B38773
:10348000E70217D501001305A513CE853E95EFD0B1
:10349000AF8997D70100938767019C435854DC5745
:1034A00063F5E70099C085479CC06244F240D2446E
:1034B000B2494A85424905616FD0CF8073700430AC
:1034C00001A09305840117D501001305651EEFD0F7
:1034D000AF85C1B7AA8729C57370043017D701001B
:1034E000130707FB14439DE2F04F8946014563151E
:1034F000D60023AE070405451C4381CB97D70100B6
:103500009387C7FA9843784315E3828097D60100E2
:103510009386C6F9904294427442850674C2E9B714
:1035200097D70100938787F89C437DB798439443CE
:103530007C43FD177CC3FC42E9FB7360043082804E
:103540005D71A6C24EDE52DC56DA5AD85ED686C609
:10355000A2C4CAC062D466D26AD097D90100938946
:10356000E9F517DB0100130BABF497D4010093844A
:1035700064F497DA0100938A2AF4054AA54B83A7DD
:1035800009009843630B0712DC4703A90700EFE02B
:10359000EFF6EFE0AFF783270B002A8C6369F50A9B
:1035A00097D7010023A6A7F00146637B251B88401F
:1035B000B3058941EFD0FFBDEFE05F99630B0512C2
:1035C0008840814601468A85EFD00FEC4DD982476D
:1035D000224463DA07009247B245228582978247E8
:1035E000E3C007FE22445C4889C713054400EFC0CE
:1035F0003FF8EFE0AFF183270B002A8C6360F50AF8
:10360000824717D70100232587EBE3EBFBFAB317BB
:10361000FA0013F70721631F072013F7770C6314D1
:10362000071C93F70702C9DF2285EF00101A49BF74
:10363000DC47C04783AC0700130944004A85EFC04C
:103640003FF35C50228582975C4C6387470B83A7CE
:103650000900984371FF03A70A0097D6010023A928
:1036600086E597D6010023A9F6E497D7010023A7A2
:10367000E7E4EFE0BF8DA9B7DC4703A9C70003ADBE
:103680000700930C49006685EFC09FEE832749022F
:103690004A8582978327C9016386470983A7090062
:1036A000984379FB03A70A0097D6010023A6F6E00A
:1036B00097D7010023A4E7E0A1B7EFE02FE4EFE004
:1036C000EFE483270B002A8CE363F5F883A70A0055
:1036D000884001499043B305894117D70100232948
:1036E00087DD13361600EFD0DFAAEFE03F86E3193F
:1036F00005ECEFC0BFD1E9B51C4CCA85E69763EA7B
:10370000FC049C4089CF02C866CA22CCEFF0CFE609
:103710008840814601460C08EFD0EF860DF97370A2
:10372000043001A083278901E685EA97636CFD04D4
:103730009C4089CF02C86ACA4ACCEFF0EFE38840C8
:10374000814601460C08EFD00F8429F973700430CC
:1037500001A003A509005CC000C8EFC07FDEC5BDA5
:10376000EFE0CFFE83A70900DC47C047930C44007D
:103770006685EFC0FFDF5C4C638F47015C5022859C
:1037800082973DBD03A509002322F90023282901C2
:10379000EFC01FDB21B71C4C00C83307F90058C02D
:1037A000636DEC02330C2C416363FC029C4089CFB7
:1037B00002C84ACA22CCEFF02FDC8840814601467D
:1037C0000C08EFC05FFC5DF97370043001A003A525
:1037D0000A00E685EFC0DFD655B703A50900E685E8
:1037E000EFC01FD661BF9247144C00C83387D70083
:1037F00058C0636FEC06B307FC4063E4D7065C5027
:10380000228582975C4CE39D47DB144C924798409D
:10381000B69711CF02C83ECA22CCEFF0EFD5884050
:10382000814601460C08EFC01FF6E31B05D87370F4
:10383000043001A092471CCC95C3E2975CC000C83D
:10384000930544006367FC0003A50A00EFC05FCF47
:1038500085BB03A50900EFC0BFCE9DB373700430D4
:1038600001A003A50A0093054400EFC07FCD89BBEA
:103870006374FC00E375F7F803A5090093054400A1
:10388000EFC01FCC35BB411122C406C626C24AC0B8
:1038900017D40100130404C2EFF0CFE21C4095CB13
:1038A000EFF08FE41C409DC38148014881470947E0
:1038B00081461306004097D50100938525B0170572
:1038C0000000130525C8EFD0FF9939E97370043063
:1038D00001A017D90100130969E14A85EFC03FC370
:1038E00097D401009384C4E12685EFC05FC20146EE
:1038F000C145114597D7010023A227BD97D70100E5
:1039000023AC97BAEFC09FDB17D701002324A7BAD7
:1039100011CD97D501009385E5A9EFD04FFC49B7AC
:10392000B2402244924402494101828073700430C3
:1039300001A0A5C9797156CAAA8A1305C00222D46A
:1039400026D24AD04ECE52CC06D65AC85EC63A8946
:10395000B689328AAE84892B2A8405C9EFF08FD6C6
:1039600097D70100938707B59C439DCFEFF0CFD742
:10397000130544002320540104CC232E44012320AA
:10398000340323222403EFC0DFB92285B25022542E
:1039900092540259F249624AD24A424BB24B4561B3
:1039A00082807370043001A097DB0100938B0BD4ED
:1039B0005E85EFC0DFB517DB0100130B6BD45A85B2
:1039C000EFC0FFB40146C145114597D7010023A7B9
:1039D00077AF97D7010023A167AFEFC03FCE17D7CE
:1039E00001002329A7AC01C997D501009385859CC7
:1039F000EFD0EFEEA5BF7370043001A039C50111FF
:103A000022CC06CE26CA17D401001304A4AA832808
:103A100004002A88014563850802BA842EC03687CF
:103A200032C242C4954663C5B602EFF0EFB489478F
:103A3000630BF5020840814601468A85EFC0BFD47A
:103A4000F2406244D244056182807370043001A068
:103A50008A8581463A864685EFD02F88F2406244B7
:103A6000D244056182800840814626868A85EFC05F
:103A70009FD1F9B719C1084182807370043001A049
:103A800001E57370043001A0411106C622C42A84E6
:103A9000EFF04FC348483334A000EFF0EFC4228565
:103AA000B24022444101828001E57370043001A0DC
:103AB000411122C42A8406C6EFF0CFC00050EFF0B7
:103AC000AFC2B240228522444101828001E5737079
:103AD000043001A0411122C426C22E84AA8406C645
:103AE000EFF04FBE80D02244B240924441016FF0CB
:103AF000AFBF011106CE97D701009387A79B2AC2BB
:103B00008843B6872EC432C68A853E868146F957D9
:103B10003EC0EFC09FFCF2400561828097D7010054
:103B20009387479983A80700639508007370043052
:103B300001A00111B2872E872A8836868A8546859C
:103B40008146FD5806CE46C042C23AC43EC6EFC0CA
:103B50009FC3F2400561828001C9B70700FFED8F66
:103B600099C77370043001A07370043001A0411133
:103B700022C426C206C62A84AE84EFF0AFB4184031
:103B800093C7F4FFF98F1CC02244B2409244410114
:103B90006FF08FB509C9370700FFB3F7E50099C784
:103BA0007370043001A07370043001A06F20006EA8
:103BB0004111714522C406C6C52C2A8411C5232093
:103BC00005001105EFC0BF942285B2402244410197
:103BD000828001CDB70700FFED8F81C7737004307D
:103BE00001A099E57370043001A07370043001A046
:103BF000011122CC4AC84EC652C456C206CE26CAAD
:103C0000BA893689B28A2E842A8AEFF0EF9611E5B6
:103C1000638509007370043001A0EFE02F8E8324C8
:103C20000A00B37794006316090295C763870A00F8
:103C30009347F4FFE58F2320FA00EFE02FB1F24025
:103C4000624426854249D244B249224A924A0561D9
:103C50008280E30DF4FCE38209FEB3355001E205F6
:103C600063050900B7070004DD8D4E86C18D13057D
:103C70004A00EFE09FDAEFE06FAD19E1EFC00FF916
:103C8000EFF06FA993176500AA8963D80700B704FE
:103C90000001FD14B3F499005DB7EFF0AFA28329E2
:103CA0000A00B3773401631E090089CB63880A00D8
:103CB0009347F4FFB3F737012320FA00EFF0CFA2C8
:103CC000F9B7E31DF4FEDDB701C9B70700FFED8FBB
:103CD00099C77370043001A07370043001A04111C2
:103CE00022C42A8406C626C24AC02E89EFF08F9DC0
:103CF00004409345F9FFB3F795001CC0EFF0CF9E49
:103D0000B2402244268502499244410182802E8697
:103D10008146AA8517050000130545E4D9BB41116A
:103D200022C42A8406C6EFC04FFA0040EFC08FF9C4
:103D3000B240228522444101828009C9370700FF31
:103D4000B3F7E50099C77370043001A073700430B5
:103D500001A06F20A053B70700FFF18F81C77370D8
:103D6000043001A001E67370043001A0011122CCDF
:103D70004AC84EC652C406CE26CA3689AE892A8A99
:103D80003284EFE07FFF21E16305090073700430A6
:103D900001A0EFD0BFF683240A00CE855285B3E49C
:103DA0009900613FB37794006307F40683240A0007
:103DB000EFE0CF99F240624426854249D244B249AD
:103DC000224A05618280EFD07FF383240A00CE85EA
:103DD0005285B3E434019537B3F78400638D8702CD
:103DE000E30609FCB70500054A86C18D13054A00A4
:103DF000EFE0BFC2EFE08F9519E1EFC02FE1EFF0E8
:103E00008F9193176500AA8463DF0700B70700014D
:103E1000FD17FD8C45B783270A001344F4FFE18F9B
:103E20002320FA0071B7EFF0EF8983240A00B377FB
:103E30009400639787009347F4FFE58F2320FA00EF
:103E4000EFF08F8AE1B7411122C406C62A8426C248
:103E5000EFD0DFEA5C4085C308489304C4006316D2
:103E6000950015A0084863009502B7050002EFE031
:103E7000DFD75C40E5FB2285892A2244B240924488
:103E800041016FE0AF8C7370043001A0B2862E86C2
:103E9000AA8517050000130525D06FF09FC519C12D
:103EA000084D828001458280411122C406C62A84C1
:103EB000EFD0DFE497C70100938787609C43A1EBB5
:103EC000E56717D7010013072785F11797C601008B
:103ED00023AEE65E17C701002328F75E17D701005F
:103EE000232EF78297C701009387C75D17D701007C
:103EF0002324F782854717C70100232B075C17C7C8
:103F000001002321075C17C70100232BF75A19E88A
:103F1000EFE0CF83EF10E00701442285B240224456
:103F2000410182801305840093773500C1EFE56776
:103F30001307F5FFE917E3EDE7FC97C60100938649
:103F4000E6589C4229A0984311C7BE86BA87D84339
:103F5000E36BA7FE17C701001307C756E38AE7FA0A
:103F6000984341461384870098C2D843B306A740BC
:103F70006378D6023388A7002322D800C8C38325DC
:103F8000480097C601009386665411A0BA869842ED
:103F90005043E36DB6FE2320E80023A00601D8437A
:103FA00097C701009387C7569C43998F17C7010095
:103FB0002320F756EFD09FF931DC2285B24022440E
:103FC00041018280719911059DB729C9411122C40F
:103FD00006C62A84EFD09FD2930584FF0326C4FF30
:103FE00017C701001307874E11A03E871C43D44317
:103FF000E3EDC6FE232CF4FE0CC397C701009387A4
:10400000275198438327C4FF2244B240BA9717C769
:104010000100232FF74E41016FD05FF3828097C7D5
:1040200001009387E74E8843828082803367B50022
:104030000D8BAA871DE79308D6FFAA982A87AE861C
:104040006371150303A8060011079106232E07FFCD
:10405000E36A17FF9347F5FFC697F19B9107BE955B
:10406000AA972A9663F3C70A9386450013884700E8
:10407000B3B6D70033B8050133E7F50093C6160091
:10408000134818000D8BB3E6060113371700758F20
:10409000330EF6409386170029CF1337AE0031EB6D
:1040A00013532E002E88BE8601478328080005077B
:1040B000110823A016019106E36967FE1377CEFF6E
:1040C000BA95BA976302EE0483C6050013871700FA
:1040D0002380D700637AC70283C6150013872700A1
:1040E000A380D7006372C70203C725002381E700BE
:1040F0008280B307F640AE97850503C7F5FF8506B6
:10410000238FE6FEE39AF5FE82808280B367C500C6
:104110008D8BB308C500E9C36371150FB307A040C9
:104120008D8B13873700954693F5F50F130815000F
:104130003383A8407D166373D70015476363E60C8D
:10414000D5CF2300B5000547638DE700A300B50078
:104150000D47130825006396E70013083500230177
:10416000B500139685004D8E13970501518F3303CB
:10417000F34093968501D98E13562300AA970147E1
:1041800094C305079107E36DC7FE1377C3FFB30719
:10419000E8006307E3062380B70013871700637CFA
:1041A0001703A380B70013872700637617032381C3
:1041B000B7001387370063701703A381B700138715
:1041C0004700637A17012382B7001387570063748F
:1041D0001701A382B700828093F5F50F139785002E
:1041E000D98D139705014D8FE37715FFAA879107A6
:1041F00023AEE7FEE3ED17FF828082802A8895B721
:104200008280AA8749BF834705002A8799C7050589
:1042100083470500EDFF198D8280014582800505E9
:104220008347F5FF850503C7F5FF91C7E389E7FEDF
:104230003385E74082808147E5BFAA87850503C7AC
:10424000F5FF8507A38FE7FE75FB82808346050097
:10425000930700026397F600050583460500E38D8A
:10426000F6FE938756FD93F7D70F85C7AA8781453A
:1042700085CE01458507138606FD1317250083C6E5
:1042800007003A9506053295F5F699C13305A04029
:104290008280938536FD8346150093B515009307FC
:1042A0001500E1FA0145D5B7014582809C41238084
:1042B000A7009C4185079CC1828097C60100938618
:1042C00066219C42175703001307C7471386170040
:1042D000BA972380A70097C5010023ADC51EA94743
:1042E0006308F500930700046305F600014582802A
:1042F00075DE370610F005078347F7FF2320F6F039
:104300009C42FD1797C5010023A6F51CEDF701455A
:1043100082804D712322911423202115232A5113C9
:10432000232481132326111423248114232E3113D3
:10433000232C411323286113232671132322911365
:104340002320A113232EB111AA842E8932C6130C67
:104350005002A54A8347090063808703B9CB804098
:1043600011A0A1CB2300F40080400509050480C002
:1043700083470900E39787FF034619009308190054
:10438000C686130D0002FD597D5A014813055005DC
:104390009307D6FD93F7F70F138916006363F52A89
:1043A00017C70100130707C68A07BA979C43BA9735
:1043B00082878320C1140324811483244114032998
:1043C00001148329C113032A8113832A4113032B68
:1043D0000113832BC112032C8112832C4112032D54
:1043E0000112832DC11171618280A14C02C48547E5
:1043F00063D50715B2478040938B770093F68BFF08
:1044000003AB060083A94600938786003EC66686F6
:1044100081465A85CE85EF10302A2AC881476385A8
:104420003723930D4101854B668681465A85CE859B
:10443000EF10A072814666862A8BAE89EF10D027D6
:10444000A24723A0AD0093861B00910D6384370122
:10445000B68BD9BFE37E9BFF63DD4601A287238035
:10446000A70180407D1A930714009CC03E84E3C8D6
:1044700046FF93962B001C08BE9631A893877705BC
:104480002300F4008040FD1B93871B00050480C0BF
:10449000F116E351F0EC9C42E3E2FAFE9387070346
:1044A000C5B79C409306000332472380D7009C4049
:1044B00093064700C14C1386170090C0130680076F
:1044C000A380C700804002C4BA87050480C003AB44
:1044D0000700814936C625BFB24783AC0700938BDE
:1044E000470063840C1C635F40199307D002631973
:1044F000FD1683C70C0085C363DC09189440850C46
:104500007D1A2380F6008040050480C083C70C001C
:10451000E5F7635D40018040930700022300F4004B
:1045200080407D1A050480C0E31A0AFE5EC61DB5F0
:1045300002C48547A94CE3CF07EBB247804093867E
:10454000470071B703C61600CA8699B59C4093060A
:1045500050022380D7008040050480C0E5BBC14CD9
:1045600002C471B5B24703C61600CA8683A9070004
:1045700091073EC6E35E0AE04E8AFD5911BD03C6AF
:104580001600130DD002CA8621B59347FAFFFD87A6
:1045900003C61600337AFA00CA86DDBB03C61600CE
:1045A000130D0003CA86EDB383C51600930906FDFB
:1045B000CA86938705FD2E86E3EEFAFA93972900C3
:1045C000BE9985068609AE9983C50600938909FDC3
:1045D000938705FD2E86E3F3FAFE69BF32479C40C0
:1045E000144311073AC62380D7008040050480C0D9
:1045F00095B3854763D3070BB24793867700E19A5B
:10460000938786003EC683A946009C4263DC090A64
:1046100094401306D002B307F0402380C6008040C8
:10462000B336F000B3093041050480C03E8BB38936
:10463000D940A94C02C4E1BB03C616000508CA86CE
:1046400081BB9C40468921B7E37D9BDD8547814B3B
:104650008546E3C547E131BD97CC0100938C8CD6EC
:10466000CE856685EF104015330AAA40635C400191
:1046700080402300A40180407D1A050480C0E31A15
:104680000AFE014A83C70C00E38207EAE3C809E691
:10469000FD197D57E394E9E6ADBDB2479386470027
:1046A0009C4336C693D9F74195B7635640019307AB
:1046B000D002E313FDFA97CC0100938CACD09307A2
:1046C00080021DBD3E8BA94C02C4804089B34D7150
:1046D000232E3113B70900409387F9FF2324811457
:1046E00023229114232C4113232A5113232611141E
:1046F00023202115232861132326711323248113DA
:10470000232291132320A113232EB1112A8A2EC410
:1047100017C40100130404DC975A0300938A8A0229
:1047200097C40100938484A33EC693055002294593
:1047300013080004B70610F083470A006386B70425
:10474000C1C71840050A13061700569797C80100FD
:1047500023A2C8D82300F7006382A706E31E06FD44
:1047600017570300130707FE05078347F7FF23A02A
:10477000F6F01C40FD1717C60100232DF6D4EDF707
:1047800083470A00E39EB7FA83461A0013051A000E
:104790002A87930B00027D5B7D5C014893055005E1
:1047A000A5489387D6FD93F7F70F130A170063E721
:1047B000F5348A07A6979C43A6978287175703006C
:1047C000130747F855F28DBF8320C11403248114C9
:1047D00083244114032901148329C113032A81135B
:1047E000832A4113032B0113832BC112032C811243
:1047F000832C4112032D0112832DC111716182801E
:10480000A14C014D854763DB0719A2479D07E19B3A
:1048100083AD070003AB4700138787003AC4668661
:1048200081466E85DA85EF1020692AC863066D35EA
:10483000130941018549668681466E85DA85EF1048
:10484000C03166868146AA8D2E8BEF10E06623204C
:10485000A90085091109E3106DFFE3FE9DFD130614
:104860000004B70610F063D189031C4013871700BA
:10487000D69797C5010023AFE5C423807701630C69
:10488000C7047D1CE3C389FFB2476800A548B3860F
:10489000F9008A061C08BE9629481303000437064F
:1048A00010F0E384A6E89C429305000363F4F8004B
:1048B000930570051840AE9793051700569717CECD
:1048C00001002329BEC02300F7006380072B638CFF
:1048D0006526F116F9B7175703001307A7E6050772
:1048E0008347F7FF23A0F6F01C40FD1797C5010092
:1048F00023A2F5BEEDF77D1C71B71C401306000422
:104900001387170097C5010023A6E5BCB386FA00FC
:10491000930500032380B6006300C73E890797C64E
:10492000010023A9F6BA5697930680072300D70003
:1049300017570300130707E1B70610F0639EC7007F
:1049400005078347F7FF23A0F6F01C40FD1717C6A5
:1049500001002321F6B8EDF7A247C14C014D9107A4
:104960002247014B832D07003EC455BDA24783ACAF
:10497000070013894700638F0C3A63548021930723
:10498000D002639EFB2E03C70C00BA85631007207C
:1049900025AC8547A94C014DE3C907E7A24791071C
:1049A000C1B7A24783461700528703AB07009107A0
:1049B0003EC4E3580CDE5A8C7D5BE5B3834617009A
:1049C000930BD0025287F1BB9347FCFFFD878346D0
:1049D0001700337CFC005287E9B383461700930B22
:1049E000000352877DBB03461700138B06FD5287D9
:1049F000930706FDB286E3EEF8FA93172B00DA97D9
:104A000005078607B29703460700138B07FD930738
:104A100006FDB286E3F3F8FE69BFA2451C402946B5
:104A2000984193861700D69717C501002324D5AA6D
:104A30002380E700138945006301C72A9307000418
:104A40006387F6204AC4D5B1854763DF0729A247AB
:104A500013877700619B930787003EC4032B4700B1
:104A60001C43635B0B3018401306000493061700C9
:104A700097C5010023A0D5A656979305D002230021
:104A8000B7006388C62CB307F0403337F000330B10
:104A90006041BE8D330BEB40A94C014D49B38346B9
:104AA000170005085287F5B9834617005287D5B914
:104AB0001C40930600041387170017C60100232B20
:104AC000E6A0D697130650022380C700E31FD7C481
:104AD00017570300130707C7B70610F005078347EA
:104AE000F7FF23A0F6F01C40FD1717C60100232393
:104AF000F69EEDF71DB9C14C014D29B31C4093063C
:104B000000042A8A1387170017C601002324E69C95
:104B1000D697130650022380C700E318D7C0175753
:104B20000300130727C2B70610F005078347F7FFF6
:104B300023A0F6F01C40FD1717C60100232CF698A1
:104B4000EDF72A8ADDB6175703001307A7BF05073D
:104B50008347F7FF2320F6F01C40FD1797C501009F
:104B600023AAF596EDF7F1162DBB1757030013078F
:104B700067BDF1FDF11635B3E3FC9DCB8549C5B1A9
:104B8000014C03C70C00BA85E30E07EAFD5829451E
:104B900013080004B70610F063570B0A1C40138675
:104BA0001700D69717C301002326C3922380E7007E
:104BB0006384A50663040609850C03C70C007D1CED
:104BC000BA8579FBE35080E91C4093050002130687
:104BD0000004B70610F021A07D1CE3050CE6138746
:104BE0001700D6972380B70017C501002324E58E50
:104BF000BA87E313C7FE175703001307A7B40507C7
:104C00008347F7FF23A0F6F01C40FD1717C50100EE
:104C10002322F58CEDF7C9B717570300130787B2A6
:104C200041DE05078347F7FF23A0F6F01C40FD1780
:104C300017C601002320F68AEDF7BDBF1757030002
:104C4000130747B0F9BF7D1BE31A1BF5A5BF175724
:104C50000300130727AFB70610F005078347F7FFD8
:104C600023A0F6F01C40FD1717C601002324F6868A
:104C7000EDF74AC45DBC97BC0100938CAC74DA8537
:104C80006685EF007033330CAC40E35C80EF1C4072
:104C900013060004B70610F021A07D1CE3020CEE01
:104CA00013871700D6972380770197C5010023A3A8
:104CB000E582BA87E313C7FE17570300130787A8D7
:104CC00005078347F7FF23A0F6F01C40FD1797C5A3
:104CD000010023A1F580EDF7C9B7175703001307AB
:104CE00067A6B5FA4AC491B4A247138747009C430C
:104CF0003AC413DBF741B5B317570300130787A472
:104D0000B70610F005078347F7FF23A0F6F01C4015
:104D1000FD1717B60100232FF67AEDF7854717B771
:104D200001002329F77A9307800717570300230B05
:104D3000F7A01DB1635680019307D002E39DFBF2FB
:104D400097BC0100938C0C681307800293058002C6
:104D500035BD975603009386E69E370610F085060C
:104D600003C7F6FF2320E6F018407D1797B5010032
:104D700023A2E5766DF701BBBE8DA94C014D45B46C
:104D8000B70710F023A0A7F201A039711303410265
:104D90002ED29A8506CE32D436D63AD83EDA42DCC6
:104DA00046DE1AC62D32F2400145216182805D71D6
:104DB0001303810322D42AC632DC2A841A866800AF
:104DC00006D6BEC236DEBAC0C2C4C6C61ACEEFF020
:104DD0004FD4B247238007003245B250018D225490
:104DE00061618280B70710F083A647F403A607F439
:104DF00003A747F4E31AD7FE8566938606FAB296B0
:104E000033B6C600B305E60023A4D7F423A6B7F44F
:104E10008280B70710F003A747F403A607F483A620
:104E200047F4E31AD7FE8566938606FAB29633B640
:104E3000C60023A4D7F4B305E60023A6B7F493076E
:104E4000000873A047308280411122C406C6514435
:104E50007D14EF00D0006DFCB240224441018280FD
:104E6000411122C406C697B701009387276717B47C
:104E700001001304646698431C401306F07C9306FB
:104E800047069387470697B5010023A9D56497B5D0
:104E9000010023A3F5646346D600B24022444101D9
:104EA00082801307478997B7010023A9E762EF00C3
:104EB00010098547631FF500184085679387F776CB
:104EC0000145E3DCE7FC6D3D2244B24041016FC087
:104ED000FFE117B501001305654F453D09454D3507
:104EE0002244B24041016FC07FE017B501001305B5
:104EF000654F61BD17B501001305454F6FF0FFE821
:104F0000411122C426C206C6856417B401001304E9
:104F1000644E938784380100FD17F5FF2285EFF07A
:104F2000DFE6C5BF411106C622C4EF0000671707C0
:104F300000001307A7F1814605469305200317B526
:104F400001001305A54BEFE0DF9E2A84EFC01FDCB4
:104F50002A8622852244B240014781468545410187
:104F60006FE0DFA9411106C6EF00607D054781476C
:104F70006316E500B2403E854101828017B501000D
:104F80001305C544EFF07FE0B24089473E854101FB
:104F900082807370043001A082807370043001A09D
:104FA000411126C24AC006C622C42A89EFD01FDC9E
:104FB00097B70100938747549C4395446387A7069E
:104FC00017B401001304C4530145EFD09F83084078
:104FD0007D5781460546A685EFE0BFBF75F525A044
:104FE000EFD03F820840FD563D46CA85EFE0BFD670
:104FF0003D897D5785460146BD45631D95020840A4
:10500000EFE03FBD0DE50145EFD0AFFF0840FD5695
:105010003D46CA85EFE03FD49374F500BD47014596
:10502000E380F4FC7370043001A08D4451BF7370B1
:10503000043001A07370043001A0011122CC4EC6CF
:1050400052C406CE26CA4AC817B401001304444B02
:1050500097B901009389494B130AF00F0145EFD02E
:105060004FFA08407D57854605468945EFE07FB6F3
:105070002A8908407D57854601469305200AEFE0BE
:105080005FB51375250A9307200A85446304F50C60
:105090000145EFD00FF708407D578546054693053B
:1050A000200AEFE01FB36303450185440145EFD0BB
:1050B0004FF50840FD563D468945EFE0DFC93D8983
:1050C000BD476303F500854408408145EFE0FFC616
:1050D00025C5084081458544EFE01FBF0145EFD05D
:1050E0004FF20840FD563D468945EFE0DFC63D8959
:1050F000BD476303F500854408408145EFE0FFC3E9
:1051000019C908407D5785460146BD45EFE07FAC93
:105110007370043001A008407D5785460146BD45A7
:10512000EFE03FAB75F5EDF483A70900850717B7EE
:105130000100232BF73C1DB708408145EFE0DFB8A5
:1051400019ED91EC83A70900850717B70100232DFE
:10515000F73A69B79304E9F5B334900015BF854475
:10516000B5BF79714AD006D622D426D24ECE52CCC3
:1051700056CA5AC85EC662C466C26AC02A89EFE0CF
:105180003FA397B7010023ADA7366300054017BAC8
:105190000100130A6A3603250A0097B901009389B2
:1051A00069350544EFC0CFD2AA8403A50900EFC03A
:1051B0002FD28D47630EF53CA14B854A97B4010071
:1051C00093840434094B0D4C03250A00EFC00FF5FE
:1051D00003A50900EFC08FF403250A00EFC04FCFED
:1051E00063036501054403A50900EFC06FCE6303A7
:1051F000650105448840D685EFE03FB493F73A0057
:1052000003250A0063950734EFC08FCC6303650163
:10521000054493F75A0003A5090063950732EFC0D0
:105220002FCB630365010544FD1B860AE39E0BF843
:1052300003250A0017BD0100130D4D2D894AEFC04B
:10524000EFED03A50900854B930C000AEFC00FEDAD
:1052500088400D4B130CD005EFE0FFBEEFE05F95EB
:1052600097B7010023AEA728630E05304A85EFC02B
:10527000EFEA4A85EFC0CFC5630355010544884076
:105280009305200AEFE07FAB884001478146014645
:105290009305F00FEFE0FF936303950105444A8502
:1052A000EFC00FC363035501054488409305D00F39
:1052B000EFE0BFA888400147814601469305F00F03
:1052C000EFE03F919307D00F6303F50005444A8553
:1052D000EFC00FC063035501054488408945EFE0E6
:1052E000DFA54A85EFC0CFBE630365010544884052
:1052F0008145EFE09FA49307F00F6303F500054499
:1053000088408945EFE05F9C9307F00F6303F50049
:1053100005444A85EFC08FE04A85EFC06FBB630349
:105320005501054488408945EFE03FA14A85EFC01B
:105330002FBA630365010544884001478146014651
:105340009305F00FEFE0FF88630385010544884073
:105350009305F00FEFE05F976303850105448840F4
:105360008145EFE07F9611C105444A85EFC04FB6F5
:1053700063036501054403250A00EFC06FB56303AD
:105380006501054403A50900EFC08FB463036501FF
:1053900005448840B945EFE05F9A8840FD560546D0
:1053A0008545EFE05F9B058911E105448840814513
:1053B000EFE09F91B9476303F50005448840B94584
:1053C000EFE09F9088408145EFE01F9011C10544B8
:1053D0004A85EFC0AFD403250A00EFC02FD403A540
:1053E0000900EFC0AFD34A85EFC08FAE630355010C
:1053F000054403250A00EFC0AFAD63035501054422
:1054000003A50900EFC0CFAC6303550105448840F4
:10541000FD563D468545EFE01F943D89BD4763033A
:10542000F500054488408145EFE01F8A11C105441D
:105430004A85EFC0EFA963036501054403250A000F
:10544000EFC00FA963036501054403A50900EFC080
:105450002FA86303650105444A85EFC02FCC0325BF
:105460000A00EFC0AFCB03A50900EFC02FCB4A85E0
:10547000EFC00FA663035501054403250A00EFC0E2
:105480002FA563035501054403A50900EFC04FA4F0
:1054900063035501054489450145EFC00FB68840B7
:1054A000FD563D468545EFE01F8B3D89BD476303B3
:1054B000F500054488408145EFE01F8111C1054496
:1054C0004A85EFC0EFA063037501054403250A0078
:1054D000EFC00FA063037501054403A50900EFC0E9
:1054E0002F9F63037501054401458145EFC0EFB06F
:1054F0004A85EFC0EF9D63035501054403250A006B
:10550000EFC00F9D63035501054403A50900EFC0DB
:105510002F9C6303550105448840EFE0DF924A85E4
:10552000EFC00F9B63036501054403250A00EFC02C
:105530002F9A6303650303A50900EFC06F99737089
:10554000043001A0EFC0CF98E31F85CDF1B9EFC0C3
:105550002F98E31F85CB75B903A50900EFC04F97BE
:10556000E31F65FD69FC83270D00850717B7010060
:10557000232EF7F8EFE0CFE397B7010023A2A7F8B7
:10558000E31605CE7370043001A07370043001A0DF
:105590001384D4FF3334800005B1011181480148E0
:1055A0007C00054781461306004097B501009385AE
:1055B00025E617050000130585A806CEEFB09FCAA3
:1055C000B24681480148814701471306004097B51C
:1055D0000100938565E4170500001305C5B8EFB019
:1055E0007FC88148014897B701009387E7F00547D6
:1055F00091461306004097B50100938565E21705B3
:1056000000001305259AEFB0FFC597B701009387F7
:1056100067EE814801480547A1461306004097B54B
:1056200001009385E5DF170500001305A597EFB08E
:105630007FC397B701009387E7EB9C4399CBEFE0DB
:105640002FD797B7010023ABA7EA19C5F240056130
:1056500082807370043001A07370043001A0411186
:1056600006C622C497B70100938787E89C431307B7
:105670004006850797B6010023ACF6E6638EE70087
:105680001307800C6388E7061307C0126387E702DD
:10569000B24022444101828017B40100130404E6A1
:1056A0000840EFE0CFE715CD854717B70100232F5E
:1056B000F7E2B24022444101828097B7010093870C
:1056C000E7E38843C945EFE08FE485476304F504C9
:1056D00017B70100232CF7E097B7010023AA07E0D2
:1056E00045BF08400146C945EFE04FFA8547E31D35
:1056F000F5FA79BF97B70100938747E08843EFE059
:105700000FE2C947E306F5F8854717B70100232FD5
:10571000F7DC45B797B70100938747DD9C4317B780
:105720000100232707DCADF797B70100938787DDDA
:105730009C43850717B701002326F7DC91BF17B7F5
:1057400001001307A7DC8328070097B701009387A0
:10575000A7DB0C4317B601001306C6D894431042CA
:1057600017B80100130848D80327080017B501002F
:10577000232CB5D601456306D600330717413335D0
:10578000E000904317B701001307C7D797B7010090
:10579000938707D514439C43184397B5010023A36F
:1057A000C5D4958FB337F000B307F04097B601002A
:1057B00023A8E6D27D8D8280AA95AA876385B7004B
:1057C00003C7070001E73385A74082808507FDB73F
:1057D000814863DA05003305A040B337A000B30564
:1057E000B0409D8DFD5863D906003306C040B337E5
:1057F000C000B306D0409D8E32883683AA872E879C
:10580000639F061C97B601009386C6AA63F1C50C78
:10581000416E6377C60B130EF00F6373CE00214306
:10582000335E6600F29603CE06001A9E1303000252
:105830003303C341630C0300B3956500335EC501B8
:10584000331866003367BE00B3176500135E0801A6
:10585000B355C70313150801418193D60701337669
:10586000C703B305B5024206D18E63F8B600C296EF
:1058700063E5060163F3B600C2968D8E33F7C60367
:10588000C207C183B3D6C603B306D50213150701F9
:10589000C98F63F8D700C29763E5070163F3D700A8
:1058A000C297958F33D567008145638A0800B30797
:1058B000A0403337F000B305B0403E85998D82801B
:1058C000370E00014143E36DC6F5614391BF01E628
:1058D00005483358680241676373E8081307F00FFF
:1058E00063730701214333576800BA9603C6060065
:1058F0001A96130300023303C34063190306B385EA
:1059000005419356080113150801418113D607017B
:1059100033F7D502B3D5D5024207518FB305B5028F
:105920006378B7004297636507016373B7004297D6
:10593000B305B74033F7D502C207C183B3D5D5024B
:10594000B305B50213150701C98F63F8B700C297F5
:1059500063E5070163F3B700C2978D8FA1B73707DF
:1059600000014143E361E8F86143B5BF33186800C3
:1059700033DEC500935E08013356C500B3176500DA
:105980003355DE03B39565004D8E93150801C18133
:10599000935606013377DE033385A5024207558F00
:1059A0006378A7004297636507016373A700429776
:1059B000B306A74033F7D60342064182B3D6D603D7
:1059C0004207B386D502B365C70063F8D500C29518
:1059D00063E5050163F3D500C295958D1DB7E3E638
:1059E000D5EC416863F50605930EF00F33B8DE0081
:1059F0000E0833DE060117B301001303A38B729365
:105A0000834E0300130E0002C29E330EDE41631765
:105A10000E0263E4B6006369C500B307C540958D07
:105A20003335F5003387A5403E85BA85BDBD3703C4
:105A300000014148E3EF66FA614865BF3357D6017C
:105A4000B396C601D98EB357D50133D7D501B395D7
:105A5000C501CD8F93D506013373B702139F06019D
:105A6000135F0F0113D807013316C6013315C501A3
:105A70003357B702420333680301B30FEF023A838F
:105A8000637CF80136981303F7FF6367D8006375EA
:105A9000F8011303E7FF36983308F841B37FB802E3
:105AA0003358B802C20FB3050F03139F0701135FEA
:105AB0000F0133EFEF014287637CBF00369F13076E
:105AC000F8FF6367DF006375BF001307E8FF369FC9
:105AD0004203C16F3363E3009387FFFF135806014E
:105AE000330FBF40B375F30013530301F18F3387B6
:105AF000F502B307F302B385050333030303BE9531
:105B0000135807012E986373F8007E93C167FD1741
:105B1000935508013378F80042087D8F9A95429793
:105B20006366BF00631BBF006379E5003306C740AF
:105B30003337C700958D998D32873307E54033356C
:105B4000E500B305BF40898DB397D5013357C70131
:105B500033E5E700B3D5C50189BBAE873288368708
:105B60002A836396062097A801009388A87463FE91
:105B7000C50A41676374E60A1307F00F3337C7009D
:105B80000E07B356E600B69883C60800369793060C
:105B90000002998E99CAB397D7003357E50033189E
:105BA000D600B365F7003313D50013550801B3D7FA
:105BB000A5021316080141829356030133F7A5028B
:105BC000B305F6024207D98E3E8763FCB600C29643
:105BD0001387F7FF63E7060163F5B6001387E7FF56
:105BE000C2968D8EB3F7A602420313530301B3D6B8
:105BF000A602C20733E36700B305D6023685637B8E
:105C0000B30042931385F6FF636603016374B30028
:105C10001385E6FF4207498F81454DA8B70600016D
:105C20004147E360D6F66147A9BF01E6854633D810
:105C3000C602C166637ED8089306F00F63F30601BF
:105C40002147B356E800B69883C60800BA961307F2
:105C50000002158F49E7B3870741854513560801B0
:105C60009318080193D808019356030133F7C7022C
:105C7000B3D7C7024207D98E3385F8023E8763FC4B
:105C8000A600C2961387F7FF63E7060163F5A60037
:105C90001387E7FFC296898EB3F7C60242031353F8
:105CA0000301B3D6C602C20733E36700B388D80244
:105CB0003685637B130142931385F6FF6366030108
:105CC000637413011385E6FF4207498F3A8582808A
:105CD000B70600014147E366D8F661479DB7331820
:105CE000E800B3D5D7003313E500B356D5001355FC
:105CF0000801B397E70033F7A502B3E8F60093175E
:105D00000801C18313D60801B3D5A5024207518FFC
:105D1000B386B7022E86637CD70042971386F5FFC1
:105D2000636707016375D7001386E5FF4297B306E3
:105D3000D74033F7A602C20893D80801B3D6A6020B
:105D40004207B385D702B3671701368763FCB700F4
:105D5000C2971387F6FF63E7070163F5B700138760
:105D6000E6FFC2978D8F93150601D98DC5BD63E2FD
:105D7000D514416763FEE6021308F00F3337D800ED
:105D80000E0733D8E60097A501009385A552C2956A
:105D900003C80500930500023A98B385054185E1E3
:105DA0000547E3E5F6F23335C5001347150039BF63
:105DB000B70500014147E3E6B6FC6147D9B7335761
:105DC0000601B396B600D98E93DE060133D70701DC
:105DD000B378D703B397B700335805013363F8009E
:105DE00093970601C183135803013316B600335746
:105DF000D703C20833E80801338FE7023A8E637C89
:105E0000E8013698130EF7FF6367D8006375E80161
:105E1000130EE7FF36983308E841B378D8033358B8
:105E2000D803C208B38E070393170301C183B3E7F6
:105E3000F800428763FCD701B6971307F8FF63E7C2
:105E4000D70063F5D7011307E8FFB697420EB38773
:105E5000D741C16E3367EE001388FEFF337307012D
:105E600093580701337806014182330E03033388C8
:105E7000080393560E013303C30242939A96B388E4
:105E8000C80263F30601F69813D60601B29863E0E0
:105E90001703E39317D9C167FD17FD8EC206337E42
:105EA000FE003315B500F2968145E371D5E27D170A
:105EB000A5B38145014719BDB2883687AA872E88C8
:105EC0006398061C97A601009386C63E63F8C50A30
:105ED0004163637E66081303F00F6373C3002147B9
:105EE0003353E6009A9603CE0600130300023A9E4F
:105EF0003303C341630C0300B3956500335EC501F2
:105F0000B31866003368BE00B317650013D60801E6
:105F10003377C80213950801418193D6070133589E
:105F2000C8024207D98E3308050363F80601C696F6
:105F300063E5160163F30601C696B386064133F79F
:105F4000C602C207C183B3D6C602B306D502131573
:105F50000701C98F63F8D700C69763E5170163F39C
:105F6000D700C697958F33D5670081458280370368
:105F700000014147E36666F661479DB701E60546C5
:105F8000B3581603416663F3C8081306F00F637332
:105F90001601214733D6E800B29603CE060013035C
:105FA00000023A9E3303C34163190306B3851541CA
:105FB00013D7080113950801418113D60701B3F6E1
:105FC000E502B3D5E502C206D18EB305B50263F88A
:105FD000B600C69663E5160163F3B600C696B385B0
:105FE000B640B3F6E502C207C183B3D5E502B305F7
:105FF000B50213950601C98F63F8B700C69763E52C
:10600000170163F3B700C6978D8FB1BF3706000144
:106010004147E3E1C8F86147B5BFB398680033D79B
:10602000C501B3176500335EC50113D50801B3760A
:10603000A702B3956500336EBE0093950801C18138
:1060400013560E013357A702C206D18E3387E502DD
:1060500063F8E600C69663E5160163F3E600C696AC
:106060003386E640B376A602420E135E0E01335627
:10607000A602C2063386C502B3E5C60163F8C500B1
:10608000C69563E5150163F3C500C695918D0DB7FF
:10609000E3EED5EC416763F5E604930EF00F33B7FA
:1060A000DE000E0733D3E60097A80100938888200E
:1060B0009A9883CE0800130E0002BA9E330EDE417A
:1060C00063170E0263E4B6006369C500B307C540F9
:1060D000958D3335F5003388A5403E85C28579B569
:1060E000B70800014147E3EF16FB614765BF33572F
:1060F000D601B396C601D98EB357D50133D7D50192
:10610000B395C501CD8F93D506013373B702139FA5
:106110000601135F0F0193D807013316C60133152B
:10612000C5013357B7024203B36813013308EF02C6
:106130003A8363FC0801B6981303F7FF63E7D800BE
:1061400063F508011303E7FFB698B3880841B3FF6E
:10615000B802B3D8B802C20FB3051F03139F0701DB
:10616000135F0F0133EFEF014687637CBF00369F5B
:106170001387F8FF6367DF006375BF001387E8FFCD
:10618000369F4203C1683363E3009387F8FF1358D7
:106190000601330FBF40B375F30013530301F18FB2
:1061A0003387F502B307F302B38505033303030313
:1061B000BE95135807012E986373F8004693C16784
:1061C000FD17935508013378F80042087D8F9A95A2
:1061D00042976366BF00631BBF006379E500330627
:1061E000C7403337C700958D998D32873307E54017
:1061F0003335E500B305BF40898DB397D5013357DB
:10620000C70133E5E700B3D5C5018DB397A70100FA
:106210009387C729944317A701001307E72718435B
:10622000C8C2637BE50017A701001307A72708432F
:106230008C4391056FA0CFB0411122C406C617A7A9
:106240000100130767262A8408438C439105EFA0B9
:106250002FAF97A70100938767229C436376F400D2
:1062600097A7010023AC8720B240224441018280DD
:1062700097A7010093878723984394437C43FD1796
:106280007CC3FC4299E3736004308280011122CC0C
:1062900026CA2A84AE844AC84EC652C456C206CE06
:1062A000EFB0DFA51C4003290401B7090001B3E5E5
:1062B0009700930AC4000CC08144FD19370A0002FC
:1062C0001840638C2A03032609004A85B3654701F9
:1062D000B376360193175600758F0329490063C4BE
:1062E000070001E7F1BFE39DE6FC9317760063D357
:1062F0000700D58CEFC07F8FE1B793C4F4FFF98C12
:1063000004C0EFB0BFC40840F2406244D2444249E6
:10631000B249224A924A05618280411106C622C4CE
:10632000EFE05FC017F7FFFF1307C7B381460546CD
:106330009305400617A501001305C50CEFD06FDFCC
:1063400019C92A84EFB09F9C2A860147814685455A
:106350002285EFD0AFEAEFB0EFF4B240224401451E
:0463600041018280F5
:02000004800278
:100000004445FEFF4246FEFF4C45FEFF4246FEFFD2
:100010004246FEFF4246FEFF4246FEFF6445FEFFAB
:100020004246FEFF4246FEFF7E45FEFF8A45FEFF3A
:100030004246FEFF9C45FEFFA845FEFFA845FEFF89
:10004000A845FEFFA845FEFFA845FEFFA845FEFF08
:10005000A845FEFFA845FEFFA845FEFF4246FEFF5D
:100060004246FEFF4246FEFF4246FEFF4246FEFF7C
:100070004246FEFF4246FEFF4246FEFF4246FEFF6C
:100080004246FEFF4246FEFF4246FEFF4246FEFF5C
:100090004246FEFF4246FEFF4246FEFF4246FEFF4C
:1000A0004246FEFF4246FEFF4246FEFF4246FEFF3C
:1000B0004246FEFF4246FEFF4246FEFF4246FEFF2C
:1000C0004246FEFF4246FEFF4246FEFF4246FEFF1C
:1000D0004246FEFF4246FEFF4246FEFF4246FEFF0C
:1000E0004246FEFF4246FEFF4246FEFF4246FEFFFC
:1000F0004246FEFF4246FEFF4246FEFF4246FEFFEC
:10010000DC45FEFFF245FEFF4246FEFF4246FEFF93
:100110004246FEFF4246FEFF4246FEFF4246FEFFCB
:100120004246FEFF3846FEFF4246FEFF4246FEFFC5
:10013000EA43FEFFA244FEFF4246FEFF4246FEFFA8
:10014000D844FEFF4246FEFF3045FEFF4246FEFF1A
:100150004246FEFF5E45FEFF5049FEFFA449FEFFFA
:100160005849FEFFA449FEFFA449FEFFA449FEFF33
:10017000A449FEFF4A48FEFFA449FEFFA449FEFF32
:100180006448FEFF7048FEFFA449FEFF8248FEFF60
:100190008E48FEFF8E48FEFF8E48FEFF8E48FEFF13
:1001A0008E48FEFF8E48FEFF8E48FEFF8E48FEFF03
:1001B0008E48FEFFA449FEFFA449FEFFA449FEFFAE
:1001C000A449FEFFA449FEFFA449FEFFA449FEFF87
:1001D000A449FEFFA449FEFFA449FEFFA449FEFF77
:1001E000A449FEFFA449FEFFA449FEFFA449FEFF67
:1001F000A449FEFFA449FEFFA449FEFFA449FEFF57
:10020000A449FEFFA449FEFFA449FEFFA449FEFF46
:10021000A449FEFFA449FEFFA449FEFFA449FEFF36
:10022000A449FEFFA449FEFFA449FEFFA449FEFF26
:10023000A449FEFFA449FEFFA449FEFFA449FEFF16
:10024000A449FEFFA449FEFFA449FEFFA449FEFF06
:10025000A449FEFFA449FEFFC248FEFFF048FEFF8E
:10026000A449FEFFA449FEFFA449FEFFA449FEFFE6
:10027000A449FEFFA449FEFFA449FEFF4649FEFF34
:10028000A449FEFFA449FEFFA846FEFFA247FEFFC9
:10029000A449FEFFA449FEFF1448FEFFA449FEFF47
:1002A0003A48FEFFA449FEFFA449FEFF9E49FEFF17
:1002B000000102020303030304040404040404040D
:1002C00005050505050505050505050505050505DE
:1002D00006060606060606060606060606060606BE
:1002E00006060606060606060606060606060606AE
:1002F000070707070707070707070707070707078E
:10030000070707070707070707070707070707077D
:10031000070707070707070707070707070707076D
:10032000070707070707070707070707070707075D
:10033000080808080808080808080808080808083D
:10034000080808080808080808080808080808082D
:10035000080808080808080808080808080808081D
:10036000080808080808080808080808080808080D
:1003700008080808080808080808080808080808FD
:1003800008080808080808080808080808080808ED
:1003900008080808080808080808080808080808DD
:1003A00008080808080808080808080808080808CD
:1003B000546D725100000000546D7220537663003A
:1003C000286E756C6C2900004572726F7220696E20
:1003D00020787878207461736B73200D0A00000018
:1003E0006D69616F750A00006D69616F75320A0091
:1003F00068756E6772790A0054696D657232000023
:10040000436865636B54696D657200005761697478
:100410004F0000005365744200000000526E647685
:0404200000000000D8
:100424001000000000000000017A5200017C01016C
:100434001B0D020010000000180000009053FEFF86
:100444008A03000000000000100000002C000000DF
:100454000657FEFF5E0300000000000010000000CD
:1004640040000000505AFEFF54030000000000004A
:08050C00FC8F01000900000052
:040000058000004037
:00000001FF
